:020000040800F2
:1000000000060020E1010008E3010008E301000808
:10001000E3010008E3010008E3010008E301000830
:10002000E3010008E3010008E3010008412F000894
:10003000E3010008E3010008E3010008E301000810
:10004000E3010008E3010008E3010008E301000800
:10005000E3010008E3010008E3010008E3010008F0
:10006000E3010008E3010008E3010008E3010008E0
:10007000E3010008E3010008E3010008E3010008D0
:10008000E3010008E3010008E3010008E3010008C0
:10009000E3010008E3010008E3010008E3010008B0
:1000A000E3010008E3010008E3010008E3010008A0
:1000B000E9310008E3010008E3010008E30100085A
:1000C000E3010008E3010008E3010008E301000880
:1000D000E3010008E3010008E3010008E301000870
:1000E000E3010008E3010008E3010008E301000860
:1000F000E3010008E3010008E3010008E301000850
:10010000E3010008E3010008E3010008E30100083F
:10011000E3010008E3010008E3010008E30100082F
:10012000E3010008E3010008E3010008E30100081F
:10013000E3010008E3010008E3010008E30100080F
:10014000E3010008E3010008E3010008F5260008C8
:10015000E3010008E3010008E3010008E3010008EF
:10016000E3010008E3010008E3010008E3010008DF
:10017000E3010008E3010008E3010008E3010008CF
:10018000E3010008E3010008E3010008E3010008BF
:10019000E3010008E3010008E3010008E3010008AF
:1001A000E3010008E3010008E3010008E30100089F
:1001B000E3010008E3010008E3010008E30100088F
:1001C000E3010008E3010008E3010008E30100087F
:1001D000E3010008E3010008E3010008E30100086F
:1001E00002E000F000F8FEE772B6374880F30888B6
:1001F000364880F3098836483649086040F20000E6
:10020000CCF200004EF63471CEF200010860BFF36C
:100210004F8FBFF36F8F40F20000C0F2F0004EF638
:100220008851CEF200010860BFF34F8FBFF36F8F8C
:100230004FF00000E1EE100A4EF63C71CEF20001E4
:100240000860062080F31488BFF36F8F01F01AFF57
:1002500002F014FE4FF055301F491B4A91423CBF3B
:1002600041F8040BFAE71D49184A91423CBF41F896
:10027000040BFAE71A491B4A1B4B9A423EBF51F83E
:10028000040B42F8040BF8E700201849184A914281
:100290003CBF41F8040BFAE701F0F8FE02F042FE21
:1002A000144C154DAC4203DA54F8041B8847F9E7A7
:1002B00000F042F8114C124DAC4203DA54F8041B22
:1002C0008847F9E701F0E0BE000600200022002088
:1002D0000000000808ED00E00000002000060020FB
:1002E000603500080022002040220020402200202B
:1002F000E02D0020E0010008E0010008E001000816
:10030000E00100082DE9F04F2DED108AC1F80CD066
:10031000C3689D46BDEC108ABDE8F08F002383F3CF
:1003200011882846A047002001F05CFAFEE701F0A2
:10033000EBF900DFFEE7000038B500F0A5FB01F0A7
:1003400071FE054601F094FE0446C8B90E4B9D426D
:1003500018D001339D4218BF044641F2883504BFCE
:1003600001240025002001F067FE0CB100F072F8B6
:1003700000F0EAFC284600F0BDF800F06BF8F9E761
:100380000025EFE70546EDE7010007B008B500F0EE
:100390004DFBA0F120035842584108BD07B5042188
:1003A00001900DEB010000F05FFB03B05DF804FB72
:1003B00038B5302383F31188174803680BB101F077
:1003C000DDFA164A144800234FF47A7101F0CCFA92
:1003D000002383F31188124C236813B12368013B77
:1003E0002360636813B16368013B63600D4D2B7834
:1003F00033B963687BB9022000F010FC32236360DC
:100400002B78032B07D163682BB9022000F006FC80
:100410004FF47A73636038BD40220020B1030008B6
:100420006023002058220020084B187003280CD8A5
:10043000DFE800F008050208022000F0E5BB02201A
:1004400000F0D8BB024B00225A60704758220020AF
:1004500060230020234B244A10B51C461968013143
:100460003FD004339342F9D16268A24239D31F4B83
:100470009B6803F1006303F540439A4231D20020A8
:1004800000F01CFB0220FFF7CFFF194B1A6C002273
:100490001A64196E1A66196E596C5A64596E5A6646
:1004A0005A6E5A6942F080025A615A6922F08002FB
:1004B0005A615A691A6942F000521A611A6922F0A7
:1004C00000521A611B6972B64FF0E0233021C3F865
:1004D000084DD4E9003281F311889D4683F30888E2
:1004E000104710BD00C0000820C0000800220020F6
:1004F000003802402DE9F04F93B0DFF804930290EA
:100500002022FF210AA8D9F8085000F0C7FBB34AFF
:100510001378A3B9B248012103601170302383F32B
:10052000118803680BB101F029FAAE4AAC480023E8
:100530004FF47A7101F018FA002383F31188029BBB
:1005400013B1A94B029A1A60A84A029C1378032B94
:100550001EBF00231370A44A4FF0000B18BF536056
:10056000CDF804B05E46DA46012000F04DFB24B120
:100570009D4B1B68002B00F0F981002000F056FA1B
:10058000071EF4DB012000F035FBA7F1210016283F
:10059000EAD801A353F820F0F50500081106000879
:1005A0009F0600086905000869050008690500083C
:1005B00023070008E3080008050800086108000890
:1005C00087080008AD08000869050008BF08000892
:1005D000690500082B0900087D0600086905000868
:1005E00073090008010600087D0600086905000877
:1005F000610800080220FFF7C9FE002840F0E381EF
:10060000029B7B48BBF1000F08BF1C46022140E063
:100610004FF47A7000F00AFA071EF1DB0220FFF7B0
:10062000B5FE0028ECD0013F052F00F2CE81DFE8B7
:1006300007F003070A0D10330520FFF7AFFE14E0A3
:10064000D9F80000F9E7D9F80400F6E7D9F808006E
:10065000F3E74FF01C08404600F032FA08F10408B6
:10066000FFF79CFEB8F12C0FF5D1019B012000FA99
:1006700007F71F43FBB201934FF0000A00F05AFB4B
:100680002EB1019B03F00B030B2B08BF002459482C
:10069000022100F0E9F967E7D9F80C00CDE7002E58
:1006A000AED0019B03F00B030B2BA9D10220FFF767
:1006B0006DFE07460028A3D0012000F0FFF90220BC
:1006C000FFF7B2FE00261FFA86F8404600F006FA51
:1006D000044670B10021404600F010FA01360028AF
:1006E000F1D1BB4604464448022100F0BDF93E4624
:1006F0003AE70120FFF798FE2546D9F80830AB42CB
:1007000007D9284600F0DCF9013040F0618104355A
:10071000F3E7364B00251D70334BBB465D603E460C
:10072000ACE7002E3FF46CAF019B03F00B030B2BE7
:100730007FF466AF0220FFF777FE322000F076F9F3
:10074000B0F10008FFF65CAF18F003077FF458AF74
:10075000D9F8082008EB050393423FF651AFB8F5EE
:10076000807F3FF74DAF254B0393B8450BDD4FF42A
:100770007A7000F05BF90028FFF642AF039B013767
:1007800003F8010BF0E7C820FFF700FE074600283A
:100790003FF436AF1F2D11D8C5F1200242450AABF8
:1007A00025F0030028BF424614490392184400F084
:1007B0004FFA039A1148FF2100F070FA4FEAA8039C
:1007C0000E490393C8F38702284600F06FFA0646E5
:1007D000002888D0039B05EB83054FE75C230020AE
:1007E00040220020B103000860230020582200208E
:1007F0003C32000834320008383200085C22002005
:10080000002200200220FFF7C1FD00283FF4F8AECF
:1008100000F0A0F900283FF4F3AE0027B846D9F85D
:100820000830BB4218D91F2F11D80A9B01330ED0B4
:1008300027F0030312AA134453F8203C05934046C3
:10084000042205A900F0AAFA04378046E7E73846F3
:1008500000F036F90590F2E74046FFF79FFD0DE7FF
:100860000023642105A8059300F0F4F800287FF424
:10087000C7AE0220FFF78AFD00283FF4C1AE0598FD
:1008800000F050F9E9E70023642105A8059300F082
:10089000E1F800287FF4B4AE0220FFF777FD0028CE
:1008A0003FF4AEAE059800F04DF9D6E70220FFF711
:1008B0006DFD00283FF4A4AE00F05CF9CDE7022006
:1008C000FFF764FD00283FF49BAE05A9142000F05B
:1008D00057F90390FFF762FD039905A800F0C4F8EB
:1008E000CCE6322000F0A2F8071EFFF689AEBB0767
:1008F0007FF486AED9F8082007EB0A0393423FF64F
:100900007FAE0220FFF742FD00283FF479AE27F0CA
:1009100003075744BA453FF4B1AE504600F0D0F853
:10092000FFF73CFD0AF1040AF4E74FF47A70FFF791
:100930002DFD00283FF464AE00F00CF9002849D0EA
:100940000A9B01330BD008220AA9002000F0AEF95F
:1009500000283FD02022FF210AA800F09FF91E485E
:10096000022100F081F81D4800F042FF13B0BDE8FD
:10097000F08F002E3FF444AE019B03F00B030B2BD2
:100980007FF43EAE0023642105A8059300F062F8D1
:10099000074600287FF434AE0220FFF7F7FC8046BC
:1009A00000283FF42DAE02210B4800F05DF841F223
:1009B000883000F01DFF059800F0EEF9464600F083
:1009C000B9F93C46D0E5064658E64FF0000A17E66E
:1009D000BB4688E6374686E634320008A08601002A
:1009E00070B50F4B1B780133DBB2012B0C4611D8CD
:1009F0000C4D29684FF47A730E6AA2FB033201464C
:100A000022462846B047844204D1074B00221A7080
:100A1000012070BD4FF4FA7000F0EAFE0020F8E704
:100A200010220020082600209423002007B5002370
:100A3000024601210DF107008DF80730FFF7D0FFC6
:100A400020B19DF8070003B05DF804FB4FF0FF30C4
:100A5000F9E700000A4608B50421FFF7C1FF80F05E
:100A60000100C0B2404208BD30B4054C2368DD69C6
:100A7000044B0A46AC460146204630BC604700BFE6
:100A800008260020A086010070B501F0D1F9094EBA
:100A9000094D3080002428683388834208D901F04A
:100AA000C1F92B6804440133B4F5404F2B60F2D3F5
:100AB00070BD00BF962300206823002001F066BAB5
:100AC00000F1006000F540400068704700F10060F0
:100AD000920000F5404001F0F1B90000054B1A68A2
:100AE000054B1B889B1A834202D9104401F09AB926
:100AF00000207047682300209623002038B5084D59
:100B0000044629B128682044BDE8384001F0AAB95C
:100B10002868204401F08EF90028F3D038BD00BFCA
:100B20006823002010F003030AD1B0F5047F05D23A
:100B300000F10050A0F51040D0F80038184670477A
:100B40000023FBE700F10050A0F51040D0F8100A98
:100B500070470000064991F8243033B10023086A39
:100B600081F824300822FFF7B1BF0120704700BF91
:100B70006C230020014B1868704700BF002004E080
:100B800070B5194B1D68194B0138C5F30B040844A7
:100B90002D0C04221E88A6420BD15C680A46013C3B
:100BA000824213460FD214F9016F4EB102F8016B65
:100BB000F6E7013A03F10803ECD181420B4602D279
:100BC0002C2203F8012B0A4A05241688AE4204D1D0
:100BD000984284BF967803F8016B013C02F104024D
:100BE000F3D1581A70BD00BF002004E08032000825
:100BF0006C320008022802BF024B4FF000529A618B
:100C0000704700BF00080240022802BF024B4FF4A9
:100C100000529A61704700BF00080240022801BFDD
:100C2000024A536983F4005353617047000802403D
:100C300070B504464FF47A764CB1412C254628BF56
:100C4000412506FB05F000F0D3FD641BF4E770BD01
:100C500010B50023934203D0CC5CC4540133F9E7B0
:100C600010BD000010B5013810F9013F3BB191F9FA
:100C700000409C4203D11AB10131013AF4E71AB1A4
:100C800091F90020981A10BD1046FCE70346024671
:100C9000D01A12F9011B0029FAD170470244034609
:100CA000934202D003F8011BFAE770472DE9F8439D
:100CB0001F4D144695F824200746884652BBDFF89E
:100CC00070909CB395F824302BB92022FF21484620
:100CD0002F62FFF7E3FF95F82400C0F10802A2425B
:100CE00028BF2246D6B24146920005EB8000FFF7AE
:100CF000AFFF95F82430A41B1E44F6B2082E17440B
:100D00009044E4B285F82460DBD1FFF723FF00288C
:100D1000D7D108E02B6A03EB82038342CFD0FFF7E1
:100D200019FF0028CBD10020BDE8F8830120FBE7A4
:100D30006C230020024B1A78024B1A70704700BFD8
:100D4000942300201022002010B5104C104800F011
:100D5000B5F821460E4800F0DDF82468626DD2F83F
:100D6000043843F00203C2F804384FF47A70FFF7F6
:100D70005FFF0849204600F0D3F9626DD2F80438CD
:100D800023F00203C2F8043810BD00BF4C33000842
:100D900008260020543300087047000030B5094D84
:100DA0000A4491420DD011F8013B5840082340F30A
:100DB0000004013B2C4013F0FF0384EA5000F6D1FD
:100DC000EFE730BD2083B8ED02684368114301604E
:100DD00003B118477047000013B5446BD4F894343E
:100DE0001A681178042915D1217C022912D11979A8
:100DF000128901238B4013420CD101A904F14C004C
:100E000001F0F8FED4F89444019B21790246206851
:100E100000F0D0F902B010BD143001F07BBE00002C
:100E20004FF0FF33143001F075BE00004C3001F07C
:100E30004DBF00004FF0FF334C3001F047BF0000C2
:100E4000143001F049BE00004FF0FF31143001F0C2
:100E500043BE00004C3001F019BF00004FF0FF32DC
:100E60004C3001F013BF00000020704710B5D0F8DF
:100E700094341A6811780429044617D1017C022998
:100E800014D15979528901238B4013420ED1143069
:100E900001F0DCFD024648B1D4F894444FF480736D
:100EA00061792068BDE8104000F072B910BD000003
:100EB000406BFFF7DBBF0000704700007FB5124BAF
:100EC000036000234360C0E90233012502260F4B73
:100ED000057404460290019300F1840229460096AD
:100EE0004FF48073143001F08DFD094B0294CDE96D
:100EF000006304F523724FF48073294604F14C001B
:100F000001F054FE04B070BDA0320008B10E00081C
:100F1000D90D00080B68302282F311880A7903EB9F
:100F2000820290614A79093243F822008A7912B12B
:100F300003EB820398610223C0F894140374002029
:100F400080F311887047000038B5037F044613B161
:100F500090F85430ABB9201D01250221FFF734FF72
:100F600004F1140025776FF0010100F069FC84F8AA
:100F7000545004F14C006FF00101BDE8384000F01E
:100F80005FBC38BD10B5012104460430FFF71CFFDB
:100F90000023237784F8543010BD000038B5044690
:100FA0000025143001F046FD04F14C00257701F0D6
:100FB00015FE201D84F854500121FFF705FF20463F
:100FC000BDE83840FFF752BF90F8443003F06003AB
:100FD000202B07D190F84520212A4FF0000303D899
:100FE0001F2A06D800207047222AFBD1C0E90E3301
:100FF00003E0034A82630722C2630364012070474F
:101000001122002037B5D0F894341A6811780429D9
:1010100004461AD1017C022917D1197912890123BA
:101020008B40134211D100F14C05284601F096FE89
:1010300058B101A9284601F0DDFDD4F89444019B84
:1010400021790246206800F0B5F803B030BD0000F9
:10105000F0B500EB810385B09E6904460D46FEB1F4
:10106000302383F3118804EB8507301D0821FFF737
:10107000ABFEFB685B691B6806F14C001BB101907D
:1010800001F0C6FD019803A901F0B4FD024648B184
:10109000039B2946204600F08DF8002383F3118836
:1010A00005B0F0BDFB685A691268002AF5D01B8AAA
:1010B000013B1340F1D104F14402EAE7093138B5AC
:1010C00050F82140DCB1302383F31188D4F8942404
:1010D0001368527903EB8203DB689B695D6845B155
:1010E00004216018FFF770FE294604F1140001F096
:1010F000B7FC2046FFF7BAFE002383F3118838BD02
:101100007047000001F016B8012303700023C0E906
:101110000133C36183620362C36243620363704746
:1011200038B50446302383F311880025C0E9035500
:10113000C0E90555416001F00DF80223237085F3E5
:101140001188284638BD000070B500EB81030546C4
:101150005069DA600E46144618B110220021FFF7DC
:101160009DFDA06918B110220021FFF797FD3146BF
:101170002846BDE8704001F0B7B80000826802F070
:10118000011282600022C0E90422826101F038B9B4
:10119000F0B400EB81044789E4680125A4698D401F
:1011A0003D43458123600023A2606360F0BC01F0F1
:1011B00053B90000F0B400EB81040789E46801250D
:1011C00064698D403D43058123600023A260636014
:1011D000F0BC01F0CDB9000070B502230025044633
:1011E0000370C0E90255C0E90455C564856180F803
:1011F000345001F015F863681B6823B12946204676
:10120000BDE87040184770BD0378052B10B5044643
:101210000AD080F850300523037043681B680BB177
:10122000042198470023A36010BD00000178052920
:1012300006D190F85020436802701B6803B118472C
:101240007047000070B590F83430044613B10023A5
:1012500080F8343004F14402204601F0F3F863686A
:101260009B68B3B994F8443013F0600535D0002181
:10127000204601F093FB0021204601F085FB6368C6
:101280001B6813B1062120469847062384F83430A2
:1012900070BD204698470028E4D0B4F84A30E26B8D
:1012A0009A4288BFE36394F94430E56B002B4FF01A
:1012B000300380F20381002D00F0F280092284F8CF
:1012C000342083F311880021D4E90E232046FFF750
:1012D00071FF002383F31188DAE794F8452003F0C7
:1012E0007F0343EA022340F20232934200F0C580BA
:1012F00021D8B3F5807F48D00DD8012B3FD0022BE9
:1013000000F09380002BB2D104F14C02A2630222C0
:10131000E2632364C1E7B3F5817F00F09B80B3F5FE
:10132000407FA4D194F84630012BA0D1B4F84C30C2
:1013300043F0020332E0B3F5006F4DD017D8B3F598
:10134000A06F31D0A3F5C063012B90D8636894F8E7
:1013500046205E6894F84710B4F848302046B047FD
:10136000002884D04368A3630368E3631AE0B3F5FD
:10137000106F36D040F6024293427FF478AF5C4B58
:10138000A3630223E3630023C3E794F84630012BF1
:101390007FF46DAFB4F84C3023F00203C4E90E556E
:1013A000A4F84C30256478E7B4F84430B3F5A06F66
:1013B0000ED194F8463084F84E30204600F088FF75
:1013C00063681B6813B101212046984703232370EB
:1013D0000023C4E90E339CE704F14F03A363012308
:1013E000C3E72378042B10D1302383F311882046E0
:1013F000FFF7C4FE85F311880321636884F84F501A
:1014000021701B680BB12046984794F84630002B9A
:10141000DED084F84F300423237063681B68002BF0
:10142000D6D0022120469847D2E794F848301D06CE
:1014300003F00F0120460AD500F0F6FF012804D082
:1014400002287FF414AF2B4B9AE72B4B98E700F060
:10145000DDFFF3E794F84630002B7FF408AF94F8F3
:10146000483013F00F01B3D01A06204602D501F020
:10147000A9FAADE701F09CFAAAE794F84630002BF0
:101480007FF4F5AE94F8483013F00F01A0D01B069E
:10149000204602D501F082FA9AE701F075FA97E743
:1014A000142284F8342083F311882B462A462946D7
:1014B0002046FFF76DFE85F31188E9E65DB1152240
:1014C00084F8342083F311880021D4E90E232046C8
:1014D000FFF75EFEFDE60B2284F8342083F31188CB
:1014E0002B462A4629462046FFF764FEE3E700BF65
:1014F000D0320008C8320008CC32000838B590F865
:1015000034300446002B3ED0063BDAB20F2A34D8E2
:101510000F2B32D8DFE803F0373131082232313176
:101520003131313131313737C56BB0F84A309D42F6
:1015300014D2C3681B8AB5FBF3F203FB12556DB9D5
:10154000302383F311882B462A462946FFF732FEC3
:1015500085F311880A2384F834300EE0142384F8CC
:101560003430302383F3118800231A46194620466D
:10157000FFF70EFE002383F3118838BD036C03B11F
:1015800098470023E7E70021204601F007FA0021F1
:10159000204601F0F9F963681B6813B10621204663
:1015A00098470623D7E7000010B590F83430142B85
:1015B000044629D017D8062B05D001D81BB110BD81
:1015C000093B022BFBD80021204601F0E7F900215E
:1015D000204601F0D9F963681B6813B10621204643
:1015E0009847062319E0152BE9D10B2380F83430F6
:1015F000302383F3118800231A461946FFF7DAFDDA
:10160000002383F31188DAE7C3689B695B68002BCA
:10161000D5D1036C03B19847002384F83430CEE76A
:1016200000230375826803691B6899689142FBD2A5
:101630005A68036042601060586070470023037569
:10164000826803691B6899689142FBD85A680360F5
:10165000426010605860704708B50846302383F335
:1016600011880B7D032B05D0042B0DD02BB983F3F0
:10167000118808BD8B6900221A604FF0FF33836127
:10168000FFF7CEFF0023F2E7D1E9003213605A6082
:10169000F3E70000FFF7C4BF054BD9680875186869
:1016A00002681A60536001220275D860FEF72ABEF4
:1016B0009823002030B50C4BDD684B1C87B00446E6
:1016C0000FD02B46094A684600F04EF92046FFF736
:1016D000E3FF009B13B1684600F050F9A86907B01A
:1016E00030BDFFF7D9FFF9E798230020591600080D
:1016F000044B1A68DB6890689B68984294BF00208E
:101700000120704798230020084B10B51C68D8684A
:1017100022681A60536001222275DC60FFF78EFF99
:1017200001462046BDE81040FEF7ECBD982300209E
:1017300038B5074C07490848012300252370656028
:1017400001F044FB0223237085F3118838BD00BFEC
:1017500000260020D83200089823002000F044B969
:10176000034A516853685B1A9842FBD8704700BF20
:10177000001000E08B60022308618B8208467047EE
:101780008368A3F1840243F8142C026943F8442CC3
:10179000426943F8402C094A43F8242CC26843F8B4
:1017A000182C022203F80C2C002203F80B2C044AFC
:1017B00043F8102CA3F12000704700BF1D03000860
:1017C0009823002008B5FFF7DBFFBDE80840FFF7CE
:1017D00061BF0000024BDB6898610F20FFF75CBF20
:1017E00098230020302383F31188FFF7F3BF000014
:1017F00008B50146302383F311880820FFF75AFF0C
:10180000002383F3118808BD064BDB6839B14268B9
:1018100018605A60136043600420FFF74BBF4FF01D
:10182000FF307047982300200368984206D01A685A
:101830000260506099611846FFF72CBF70470000A6
:1018400038B504460D462068844200D138BD03688F
:1018500023605C608561FFF71DFFF4E710B5036846
:101860009C68A2420CD85C688A600B604C60216066
:10187000596099688A1A9A604FF0FF33836010BDEF
:101880001B68121BECE700000A2938BF0A2170B55B
:1018900004460D460A26601901F092FA01F07EFA1C
:1018A000041BA54203D8751C2E460446F3E70A2EF6
:1018B00004D9BDE87040012001F0C8BA70BD000035
:1018C000F8B5144B0D46D96103F1100141600A2AA5
:1018D0001969826038BF0A22016048601861A8183F
:1018E000144601F05FFA0A2701F058FA431BA3429D
:1018F000064606D37C1C281901F062FA27463546B5
:10190000F2E70A2F04D9BDE8F840012001F09EBAA1
:10191000F8BD00BF98230020F8B506460D4601F03B
:101920003DFA0F4A134653F8107F9F4206D12A46CC
:1019300001463046BDE8F840FFF7C2BFD169BB6839
:10194000441A2C1928BF2C46A34202D92946FFF776
:101950009BFF224631460348BDE8F840FFF77EBFB3
:1019600098230020A823002010B4C0E903230023FB
:101970005DF8044B4361FFF7CFBF000010B5194C71
:10198000236998420DD0D0E90032816813605A6013
:101990009A680A449A60002303604FF0FF33A36102
:1019A00010BD2346026843F8102F536000220260E6
:1019B00022699A4203D1BDE8104001F0FBB9936857
:1019C00081680B44936001F0E9F92269E16992684A
:1019D000441AA242E4D91144BDE81040091AFFF7A5
:1019E00053BF00BF982300202DE9F047DFF8BC80EB
:1019F00008F110072C4ED8F8105001F0CFF9D8F8A4
:101A00001C40AA68031B9A423ED81444D5E9003210
:101A10004FF00009C8F81C4013605A60C5F80090E8
:101A2000D8F81030B34201D101F0C4F989F311881C
:101A3000D5E9033128469847302383F311886B6931
:101A4000002BD8D001F0AAF96A69A0EB04094A4535
:101A500082460DD2022001F0F9F90022D8F81030A8
:101A6000B34208D151462846BDE8F047FFF728BFEA
:101A7000121A2244F2E712EB090938BF4A462946F6
:101A80003846FFF7EBFEB5E7D8F81030B34208D080
:101A90001444211AC8F81C00A960BDE8F047FFF7FC
:101AA000F3BEBDE8F08700BFA823002098230020E4
:101AB00000207047FEE70000704700004FF0FF3045
:101AC0007047000002290CD0032904D001290748DF
:101AD00018BF00207047032A05D8054800EBC20054
:101AE0007047044870470020704700BFB0330008BB
:101AF000202200206433000870B59AB005460846DD
:101B000001A9144600F0C2F801A8FFF7BFF8431C72
:101B10005B00C5E900340022237003236370C6B262
:101B200001AB02341046D1B28E4204F1020401D856
:101B30001AB070BD13F8011B04F8021C04F8010C64
:101B40000132F0E708B5302383F311880348FFF72B
:101B500059FA002383F3118808BD00BF082600202E
:101B600090F8443003F01F02012A07D190F8452075
:101B70000B2A03D10023C0E90E3315E003F0600304
:101B8000202B08D1B0F848302BB990F84520212AF5
:101B900003D81F2A04D8FFF717BA222AEBD0FAE796
:101BA000034A82630722C26303640120704700BFB7
:101BB0001822002007B5052917D8DFE801F019160B
:101BC00003191920302383F31188104A0190012151
:101BD000FFF7BAFA01980E4A0221FFF7B5FA0D484D
:101BE000FFF7DCF9002383F3118803B05DF804FBF1
:101BF000302383F311880748FFF7A6F9F2E7302373
:101C000083F311880348FFF7BDF9EBE704330008BD
:101C1000283300080826002038B50C4D0C4C0D491F
:101C20002A4604F10800FFF767FF05F1CA0204F134
:101C300010000949FFF760FF05F5CA7204F11800AA
:101C40000649BDE83840FFF757BF00BFD02A002043
:101C500020220020E4320008EE320008F9320008A9
:101C600070B5044608460D46FFF710F8C6B2204688
:101C7000013403780BB9184670BD32462946FEF789
:101C8000F1FF0028F3D10120F6E700002DE9F84F1D
:101C900005460C46FEF7FAFF2B49C6B22846FFF769
:101CA000DFFF08B10336F6B228492846FFF7D8FF10
:101CB00008B11036F6B2632E0DD8DFF88C80DFF84D
:101CC0008C90234FDFF890A0DFF890B02E7846B9C3
:101CD0002670BDE8F88F29462046BDE8F84F01F090
:101CE000A1BA252E2BD1072241462846FEF7BAFF7E
:101CF00058B9DBF800302360DBF804306360BBF8D0
:101D00000830238107350A34E0E70822494628468F
:101D1000FEF7A8FF98B90F4BA21C197809090232E7
:101D2000C95D02F8041C13F8011B01F00F015345B3
:101D3000C95D02F8031CF0D118340835C6E704F871
:101D4000016B0135C2E700BFD0330008F93200084B
:101D5000E3330008107AFF1F1C7AFF1FD8330008F6
:101D6000BFF34F8F024AD368DB03FCD4704700BF38
:101D7000003C024008B5094B1B7873B9FFF7F0FF30
:101D8000074B1A69002ABFBF064A5A6002F188321F
:101D90005A601A6822F480621A6008BD2E2D002055
:101DA000003C02402301674508B50B4B1B7893B9F3
:101DB000FFF7D6FF094B1A6942F000421A611A6810
:101DC00042F480521A601A6822F480521A601A682B
:101DD00042F480621A6008BD2E2D0020003C0240B3
:101DE0000B28F0B516D80C4C0C4923787BB90C4D58
:101DF0000E460C234FF0006255F8047B46F8042B86
:101E0000013B13F0FF033A44F6D10123237051F84C
:101E10002000F0BD0020FCE7602D0020302D0020C8
:101E2000F4330008014B53F820007047F4330008E6
:101E30000C2070470B2810B5044601D9002010BDB6
:101E4000FFF7CEFF064B53F824301844C21A0BB9E3
:101E50000120F4E712680132F0D1043BF6E700BF3D
:101E6000F43300080B2810B5044621D8FFF778FF9B
:101E7000FFF780FF0F4AF323D360C300DBB243F4C4
:101E8000007343F002031361136943F48033136159
:101E9000FFF766FFFFF7A4FF074B53F8241000F08D
:101EA000D9F8FFF781FF2046BDE81040FFF7C2BF19
:101EB000002010BD003C0240F4330008F8B512F0D9
:101EC0000103144642D18218B2F1016F57D82D4B4D
:101ED0001B6813F0010352D02B4DFFF74BFFF32388
:101EE000EB60FFF73DFF40F20127032C15D824F0EB
:101EF00001046618244C401A40F20117B1422369CC
:101F000000EB010524D123F001032361FFF74CFF0F
:101F10000120F8BD043C0430E7E78307E7D12B69D3
:101F200023F440732B612B693B432B6151F8046B05
:101F30000660BFF34F8FFFF713FF03689E42E9D09F
:101F40002B6923F001032B61FFF72EFF0020E0E750
:101F500023F44073236123693B4323610B882B8067
:101F6000BFF34F8FFFF7FCFE2D8831F8023BADB277
:101F7000AB42C3D0236923F001032361E4E7184691
:101F8000C7E700BF00380240003C0240084908B5DE
:101F90000B7828B11BB9FFF7EDFE01230B7008BDCC
:101FA000002BFCD0BDE808400870FFF7FDBE00BF65
:101FB0002E2D002010B50244064BD2B2904200D123
:101FC00010BD441C00B253F8200041F8040BE0B2ED
:101FD000F4E700BF502800400F4B30B51C6F2404BD
:101FE00007D41C6F44F400741C671C6F44F4004455
:101FF0001C670A4C236843F4807323600244084B37
:10200000D2B2904200D130BD441C00B251F8045B02
:1020100043F82050E0B2F4E700380240007000407E
:102020005028004007B5012201A90020FFF7C2FF98
:10203000019803B05DF804FB13B50446FFF7F2FF07
:10204000A04205D0012201A900200194FFF7C4FF9E
:1020500002B010BD70470000034B1A681AB9034A5A
:10206000D2F874281A607047642D002000300240B6
:1020700008B5FFF7F1FF024B1868C0F3407008BDC8
:10208000642D002070470000FEE700000A4B0B485B
:102090000B4A90420BD30B4BDA1C121AC11E22F0D2
:1020A00003028B4238BF00220021FEF7F7BD53F830
:1020B000041B40F8041BECE7A0350008E02D0020CD
:1020C000E02D0020E02D002070B5D0E915439E687A
:1020D00000224FF0FF3504EB42135101D3F8000901
:1020E0000028BEBFD3F8000940F08040C3F80009C3
:1020F000D3F8000B0028BEBFD3F8000B40F080409F
:10210000C3F8000B013263189642C3F80859C3F8AC
:10211000085BE0D24FF00113C4F81C3870BD00001A
:10212000890141F02001016103699B06FCD4122062
:10213000FFF716BB10B5054C2046FEF7E5FF4FF044
:10214000A0436365024BA36510BD00BF682D00204E
:102150004834000870B50378012B054650D12A4B4E
:10216000446D98421BD1294B5A6B42F080025A634E
:102170005A6D42F080025A655A6D5A6942F08002E7
:102180005A615A6922F080025A610E2143205B692C
:1021900000F022FC1E4BE3601E4BC4F80038002305
:1021A000C4F8003EC02323606E6D4FF40413A36394
:1021B0003369002BFCDA012333610C20FFF7D0FADE
:1021C0003369DB07FCD41220FFF7CAFA3369002B0E
:1021D000FCDA0026A6602846FFF776FF6B68C4F895
:1021E0001068DB68C4F81468C4F81C684BB90A4B63
:1021F000A3614FF0FF336361A36843F00103A36061
:1022000070BD064BF4E700BF682D00200038024087
:102210004014004003002002003C30C0083C30C0A5
:10222000F8B5446D054600212046FFF779FFA96DFA
:1022300000234FF001128F68C4F834384FF0006665
:10224000C4F81C284FF0FF3004EB431201339F42C7
:10225000C2F80069C2F8006BC2F80809C2F8080B9E
:10226000F2D20B686A6DEB65636210231361166925
:1022700016F01006FBD11220FFF772FAD4F80038DE
:1022800023F4FE63C4F80038A36943F4402343F009
:102290001003A3610923C4F81038C4F814380A4B9A
:1022A000EB604FF0C043C4F8103B084BC4F8003B50
:1022B000C4F81069C4F80039EB6D03F1100243F45F
:1022C0008013EA65A362F8BD243400084080001042
:1022D000426D90F84E10D2F8003823F4FE6343EAC2
:1022E0000113C2F8003870472DE9F84300EB810371
:1022F000456DDA68166806F00306731E022B05EBBF
:1023000041130C4680460FFA81F94FEA41104FF015
:102310000001C3F8101B4FF0010104F1100398BF36
:10232000B60401FA03F391698EBF334E06F180566D
:1023300006F5004600293AD0578A04F158014901B0
:1023400037436F50D5F81C180B43C5F81C382B18B1
:102350000021C3F8101953690127611EA7409BB3E0
:10236000138A928B9B08012A88BF5343D8F85C20BC
:10237000981842EA034301F1400205EB8202C8F8D3
:102380005C00214653602846FFF7CAFE08EB89002F
:10239000C3681B8A43EA8453483464011E432E51A8
:1023A000D5F81C381F43C5F81C78BDE8F88305EB49
:1023B0004917D7F8001B21F40041C7F8001BD5F8D6
:1023C0001C1821EA0303C0E704F13F0305EB830374
:1023D0000A4A5A6028462146FFF7A2FE05EB49103B
:1023E000D0F8003923F40043C0F80039D5F81C3880
:1023F00023EA0707D7E700BF0080001000040002AF
:10240000826D1268C265FFF75FBE00005831436DF0
:1024100049015B5813F4004004D013F4001F0CBFB3
:1024200002200120704700004831436D49015B588C
:1024300013F4004004D013F4001F0CBF022001204D
:102440007047000000EB8101CB68196A0B681360CC
:102450004B6853607047000000EB810330B5DD68C6
:10246000AA691368D36019B9402B84BF4023136055
:102470006B8A1468426D1C44013CB4FBF3F4634363
:10248000033323F0030302EB411043EAC44343F058
:10249000C043C0F8103B2B6803F00303012B09B2C3
:1024A0000ED1D2F8083802EB411013F4807FD0F837
:1024B000003B14BF43F0805343F00053C0F8003B8F
:1024C00002EB4112D2F8003B43F00443C2F8003B58
:1024D00030BD00002DE9F041244D6E6D06EB401338
:1024E0000446D3F8087BC3F8087B38070AD5D6F82A
:1024F0001438190706D505EB84032146DB68284606
:102500005B689847FA071FD5D6F81438DB071BD548
:1025100005EB8403D968CCB98B69488A5A68B2FB49
:10252000F0F600FB16228AB91868DA6890420DD2DC
:10253000121AC3E90024302383F311880B48214683
:10254000FFF78AFF84F31188BDE8F081012303FAC5
:1025500004F26B8923EA02036B81CB68002BF3D072
:1025600021460248BDE8F041184700BF682D002011
:1025700000EB810370B5DD68436D6C692668E66029
:102580004A0156BB1A444FF40020C2F810092A68C9
:1025900002F00302012A0AB20ED1D3F8080803EBB5
:1025A000421410F4807FD4F8000914BF40F080502A
:1025B00040F00050C4F8000903EB4212D2F80009C1
:1025C00040F00440C2F80009D3F83408012202FAAE
:1025D00001F10143C3F8341870BD19B9402E84BF0E
:1025E0004020206020682E8A8419013CB4FBF6F458
:1025F00040EAC44040F000501A44C6E72DE9F843D1
:102600003B4D6E6D06EB40130446D3F80889C3F8C2
:10261000088918F0010F4FEA40171AD0D6F8103881
:10262000DB0716D505EB8003D9684B691868DA68B3
:10263000904230D2121A4FF000091A60C3F8049089
:10264000302383F3118821462846FFF791FF89F351
:10265000118818F0800F1CD0D6F834380126A64017
:10266000334216D005EB84036D6DD3F80CC0DCF853
:1026700014200134E4B2D2F800E005EB04342F4416
:102680005168714515D3D5F8343823EA0606C5F8E4
:102690003468BDE8F883012303FA04F22B8923EAA6
:1026A00002032B818B68002BD3D021462846984704
:1026B000CFE7BCF81000AEEB0103834228BF03460E
:1026C000D7F8180980B2B3EB800FE2D89068A0F178
:1026D000040959F8048FC4F80080A0EB0908984455
:1026E000B8F1040FF5D818440B4490605360C7E765
:1026F000682D00202DE9F74FA24C656D6E69AB691E
:102700001E4016F480586E6107D02046FEF764FD27
:1027100003B0BDE8F04F00F047BC002E12DAD5F848
:10272000003E98489B071EBFD5F8003E23F00303E8
:10273000C5F8003ED5F8043823F00103C5F8043885
:10274000FEF774FD370505D58E48FFF7BDFC8D48B3
:10275000FEF75AFDB0040CD5D5F8083813F0060F73
:10276000EB6823F470530CBF43F4105343F4A053AD
:10277000EB6031071BD56368DB681BB9AB6923F0DD
:102780000803AB612378052B0CD1D5F8003E7D48BA
:102790009A071EBFD5F8003E23F00303C5F8003E9C
:1027A000FEF744FD6368DB680BB176489847F30297
:1027B00074D4B70227D5D4F85490DFF8C8B10027F5
:1027C0004FF0010A09EB4712D2F8003B03F4402313
:1027D000B3F5802F11D1D2F8003B002B0DDA6289BE
:1027E0000AFA07F322EA0303638104EB8703DB6839
:1027F000DB6813B1394658469847A36D01379B688B
:10280000FFB29F42DED9F00617D5676D3A6AC2F370
:102810000A1002F00F0302F4F012B2F5802F00F05C
:102820008580B2F5402F08D104EB83030022DB68DA
:102830001B6A07F5805790426AD13003D5F81848D3
:1028400013D5E10302D50020FFF744FEA20302D511
:102850000120FFF73FFE630302D50220FFF73AFE97
:10286000270302D50320FFF735FE75037FF550AF30
:10287000E00702D50020FFF7C1FEA10702D5012025
:10288000FFF7BCFE620702D50220FFF7B7FE230761
:102890007FF53EAF0320FFF7B1FE39E7636DDFF848
:1028A000E4A0019300274FF00109A36D9B685FFA34
:1028B00087FB9B453FF67DAF019B03EB4B13D3F8A2
:1028C000001901F44021B1F5802F1FD1D3F8001970
:1028D00000291BDAD3F8001941F09041C3F8001920
:1028E000D3F800190029FBDB5946606DFFF718FC8F
:1028F000218909FA0BF321EA0303238104EB8B03FB
:10290000DB689B6813B15946504698470137CCE7BE
:10291000910708BFD7F80080072A98BF03F8018BFA
:1029200002F1010298BF4FEA182884E7023304EB52
:10293000830207F580575268D2F818C0DCF80820E7
:10294000DCE9001CA1EB0C0C002188420AD104EB4D
:10295000830463689B699A6802449A605A680244D7
:102960005A606AE711F0030F08BFD7F800808C4562
:1029700088BF02F8018B01F1010188BF4FEA1828D6
:10298000E3E700BF682D0020436D03EB4111D1F850
:10299000003B43F40013C1F8003B7047436D03EB69
:1029A0004111D1F8003943F40013C1F800397047E0
:1029B000436D03EB4111D1F8003B23F40013C1F840
:1029C000003B7047436D03EB4111D1F8003923F40C
:1029D0000013C1F80039704700F1604303F561430B
:1029E0000901C9B283F80013012200F01F039A40C5
:1029F00043099B0003F1604303F56143C3F8802161
:102A00001A60704730B5039C0172043304FB032540
:102A1000C0E90653049B03630021059BC160C0E924
:102A20000000C0E90422C0E90842C0E90A1143637A
:102A300030BD0000416A0022C0E90411C0E90A2249
:102A4000C2606FF00101FEF7FBBE0000D0E9043266
:102A5000934201D1C2680AB9181D7047002070471F
:102A600003691960C2680132C260C2691344826995
:102A70000361934224BF436A03610021FEF7D4BE81
:102A800038B504460D46E3683BB16269131D126810
:102A9000A3621344E362002007E0237A33B9294696
:102AA0002046FEF7B1FE0028EDDA38BD6FF00100D8
:102AB000FBE70000C368C269013BC360436913447C
:102AC00082694361934224BF436A43610023836266
:102AD000036B03B11847704770B53023044683F386
:102AE0001188866A3EB9FFF7CBFF054618B186F319
:102AF0001188284670BDA36AE26A13F8015BA362DD
:102B0000934202D32046FFF7D5FF002383F31188B9
:102B1000EFE700002DE9F84F04460E4617469846A9
:102B20004FF0300989F311880025AA46D4F828B05F
:102B3000BBF1000F09D141462046FFF7A1FF20B1AC
:102B40008BF311882846BDE8F88FD4E90A12A7EB69
:102B5000050B521A934528BF9346BBF1400F1BD972
:102B6000334601F1400251F8040B43F8040B914243
:102B7000F9D1A36A40334036A3624035D4E90A2331
:102B80009A4202D32046FFF795FF8AF31188BD428F
:102B9000D8D289F31188C9E730465A46FEF758F86B
:102BA000A36A5B445E44A3625D44E7E710B5029C00
:102BB0000172043303FB0421C0E906130023C0E9BA
:102BC0000A33039B0363049BC460C0E90000C0E9AF
:102BD0000422C0E90842436310BD0000026AC260DB
:102BE000426AC0E904220022C0E90A226FF0010112
:102BF000FEF726BED0E904239A4201D1C26822B969
:102C0000184650F8043B0B60704700231846FAE75B
:102C1000C368C2690133C360436913448269436175
:102C2000934224BF436A43610021FEF7FDBD0000CB
:102C300038B504460D46E3683BB123691A1DA2620C
:102C4000E2691344E362002007E0237A33B929469E
:102C50002046FEF7D9FD0028EDDA38BD6FF00100FF
:102C6000FBE7000003691960C268013AC260C269EB
:102C7000134482690361934224BF436A03610023C2
:102C80008362036B03B118477047000070B53023AF
:102C90000D460446114683F31188866A2EB9FFF764
:102CA000C7FF10B186F3118870BDA36A1D70A36AB7
:102CB000E26A01339342A36204D3E16920460439F6
:102CC000FFF7D0FF002080F31188EDE72DE9F84FE2
:102CD00004460D46904699464FF0300A8AF3118813
:102CE0000026B346A76A4FB949462046FFF7A0FF22
:102CF00020B187F311883046BDE8F88FD4E90A0780
:102D00003A1AA8EB0607974228BF1746402F1BD94F
:102D100005F1400355F8042B40F8042B9D42F9D1EE
:102D2000A36A4033A3624036D4E90A239A4204D30B
:102D3000E16920460439FFF795FF8BF3118846457A
:102D4000D9D28AF31188CDE729463A46FDF780FFAC
:102D5000A36A3B443D44A3623E44E5E7D0E9042333
:102D60009A4217D1C3689BB1836A8BB1043B9B1A0B
:102D70000ED01360C368013BC360C3691A44836902
:102D800002619A4224BF436A0361002383620123E4
:102D9000184670470023FBE700F030B94FF080433E
:102DA000586A70474FF08043002258631A6102222C
:102DB000DA6070474FF080430022DA60704700000D
:102DC0004FF0804358637047FEE7000070B51B4B1F
:102DD00001630025044686B0586085620E4600F007
:102DE000BFF804F11003C4E904334FF0FF33C4E922
:102DF0000635C4E90044A560E562FFF7CFFF2B4626
:102E00000246C4E9082304F134010D4A25658023F4
:102E10002046FEF7AFFC0123E0600A4A03750092EA
:102E200072680192B268CDE90223074B6846CDE98A
:102E30000435FEF7C7FC06B070BD00BF00260020B9
:102E40005434000859340008C92D0008024AD36AD6
:102E50001843D062704700BF982300204B6843603E
:102E60008B688360CB68C3600B6943614B69036205
:102E70008B6943620B6803607047000008B5264BFE
:102E800026481A6940F2FF110A431A611A6922F4AE
:102E9000FF7222F001021A611A691A6B0A431A635F
:102EA0001A6D0A431A651E4A1B6D1146FFF7D6FFBD
:102EB00002F11C0100F58060FFF7D0FF02F138013C
:102EC00000F58060FFF7CAFF02F1540100F5806051
:102ED000FFF7C4FF02F1700100F58060FFF7BEFF4D
:102EE00002F18C0100F58060FFF7B8FF02F1A80144
:102EF00000F58060FFF7B2FF02F1C40100F58060C9
:102F0000FFF7ACFF02F1E00100F58060FFF7A6FFDC
:102F1000BDE8084000F0EEB8003802400000024072
:102F20006034000808B500F06BF9FEF701FCFFF70C
:102F300093F8BDE80840FEF76FBE00007047000040
:102F4000EFF3098305494A6B22F001024A636833B3
:102F500083F30988002383F31188704700EF00E0B2
:102F6000302080F3118862B60C4B0D4AD96821F4E9
:102F7000E0610904090C0A43DA60D3F8FC2009492E
:102F800042F08072C3F8FC200A6842F001020A6035
:102F90002022DA7783F82200704700BF00ED00E0BE
:102FA0000003FA05001000E010B5302383F3118808
:102FB0000E4B5B6813F4006314D0F1EE103AEFF39C
:102FC0000984683C4FF08073E361094BDB6B236637
:102FD00084F30988FEF78CFB10B1064BA36110BD8A
:102FE000054BFBE783F31188F9E700BF00ED00E034
:102FF00000EF00E02F030008320300080F4B1A6CAB
:1030000042F001021A641A6E42F001021A660C4A7A
:103010001B6E936843F0010393604FF0804353228B
:103020009A624FF0FF32DA6200229A615A63DA60E4
:103030005A6001225A611A60704700BF003802408E
:10304000002004E04FF0804208B51169D3680B40BE
:10305000D9B2C9439B07116107D5302383F3118887
:10306000FEF77CFB002383F3118808BD1F4B1A6910
:103070006FEAC2526FEAD2521A611A69C2F30802A9
:103080001A614FF0FF301A695A69586100215A6974
:1030900059615A691A6A62F080521A621A6A02F019
:1030A00080521A621A6A5A6A58625A6A59625A6A8D
:1030B0001A6C42F080521A641A6E42F080521A66FC
:1030C0001A6E0B4A106840F480701060186F00F49C
:1030D0004070B0F5007F1EBF4FF48030186719674D
:1030E000536823F40073536000F086B80038024040
:1030F00000700040334B4FF080521A64324A4FF454
:10310000404111601A6842F001021A601A68910782
:10311000FCD59A6822F003029A602A4B9A6812F052
:103120000C02FBD1196801F0F90119609A601A6864
:1031300042F480321A601A689203FCD55A6F42F04A
:1031400001025A671F4B5A6F9007FCD51F4A5A60FD
:103150001A6842F080721A601B4A53685904FCD501
:10316000184B1A689201FCD5194A9A60194B1A68D3
:10317000194B9A42194B21D1194A1168194A9142A7
:103180001CD140F205121A60144A136803F00F03B1
:10319000052BFAD10B4B9A6842F002029A609A68AA
:1031A00002F00C02082AFAD15A6C42F480425A64A6
:1031B0005A6E42F480425A665B6E704740F2057266
:1031C000E1E700BF003802400070004008544007AB
:1031D00000948838002004E011640020003C024084
:1031E00000ED00E041C20F4108B5FFF72BFFBDE83D
:1031F0000840FFF7D9BE000007211C20FFF7ECBBF9
:1032000008B5FFF733FF00F00BF8FDF77BFFFDF784
:1032100053FEFFF793FEBDE80840FFF7BDBD000079
:1032200070470000034611F8012B03F8012B002A18
:10323000F9D17047121000001211000012130000A3
:1032400053544D3332463F3F3F0053544D33324683
:103250003430780053544D3332463432780053546E
:103260004D333246343436585800000001203300C4
:103270000010410001105A000310590007103100DE
:103280000000000040320008130400004A32000829
:103290001904000054320008210400005E320008C6
:1032A00000000000350E0008210E00085D0E000829
:1032B000490E0008550E0008410E00082D0E0008AA
:1032C000190E0008690E000800000000010000004F
:1032D0000000000063300000D4320008F02300201A
:1032E000002600204172647550696C6F740025429D
:1032F0004F415244252D424C002553455249414CE3
:10330000250000000200000000000000511000082D
:10331000BD10000840004000A02A0020B02A002074
:103320000200000000000000030000000000000098
:10333000011100080000000010000000C02A002059
:10334000000000000100000000000000682D0020C7
:1033500001010200B51B0008C51A0008611B000826
:10336000451B0008430000006C33000809024300BD
:10337000020100C03209040000010202010005241C
:1033800000100105240100010424020205240600A6
:1033900001070582030800FF09040100020A00007A
:1033A00000070501024000000705810240000000FF
:1033B00012000000B83300081201100102000040A2
:1033C000091241570002010203010000040309042D
:1033D00025424F4152442500466C79737061726BEF
:1033E0004634003031323334353637383941424390
:1033F000444546000040000000400000004000003E
:103400000040000000000100000002000000020077
:1034100000000200000002000000020000000200A4
:10342000000002000000000045120008FD14000822
:10343000A915000840004000C82D0020C82D00201C
:1034400001000000D82D0020800000004001000095
:10345000030000006D61696E0069646C6500000026
:103460000001802A00000000AAAAAAAA00010024E4
:10347000FFFF00000000000000A00A0000000001A3
:1034800000000000AAAAAAAA00000001FFFF000095
:103490000000000000000000000000140000000018
:1034A000AAAAAAAA00000010FFDF00000000000086
:1034B000000000000000000000000000AAAAAAAA64
:1034C00000000000FFFF00000000000000000000FE
:1034D0000000000000000000AAAAAAAA0000000044
:1034E000FFFF0000000000000000000000000000DE
:1034F00000000000AAAAAAAA00000000FFFF000026
:1035000000000000000000000000000000000000BB
:10351000AAAAAAAA00000000FFFF00000000000005
:103520000000000000000000000000000A00000091
:103530000000000003000000000000000000000088
:10354000000000000000000000000000000000007B
:10355000000000000000000000000000000000006B
:10356000510500000000000000400F0000000000B6
:10357000FF00960000000008009600000000080010
:1035800004000000CC330008000000000000000030
:10359000000000000000000000000000000000002B
:00000001FF
